:030000000201B644
:03000B000206CF1B
:0300400001FF10AD
:020043000201B8
:0300330002018047
:100100000206DF00020779000207790002072600D5
:1001100002074F0002077900020779000207790001
:1001200002077900020779000207790002077900C7
:1001300002077900020779000207710002077900BF
:1001400002077900020779000207790002077900A7
:100150000207790002077900020779000207790097
:100160000207790002077900020779000207790087
:100170000207790002077900020779000207790077
:1001800053D8EF3290E6A3E020E22A90E690E0B464
:10019000002390E691E0B41F1C759AF0759B0075E2
:1001A0009D0A759E87781FE59CF59FD8FAD2077443
:1001B0008090E691F02275816F120BC9120279309E
:1001C0000C1FE4120D314016D20B120D0990E61AE5
:1001D000740C200D027404F0120A861208F5120342
:1001E000B63006031203E130040843870100000023
:1001F000C20430080512083D80E731843007091237
:10020000087930070312077AE55754046554606291
:100210006554F554E5567050D55557755510200B5B
:100220001CE4120D31404BD20B120D0990E61A74EA
:100230000C200D027404F0120A86020272E53312D9
:100240000D156006120D27020272C20B300C1690BB
:100250000AB07401F0A3E4F0900AC674FFF0A3F0B2
:10026000A3F01203B6020272D55607E4121026124A
:100270000D27000000000021E1C206C204C205C231
:1002800000C201C20CC20D753400D20E900040E0D5
:10029000600FD20CA3E0F9A3E0C9900AB0F0A3E983
:1002A000F0755600755400755510C20B120D097487
:1002B000FF90E65DF090E65FF0754055754153752F
:0802C0004242754353E4F5537B
:1002C800F550F551F552F537F54FF55990E680E0C0
:1002D80020E70C900AB3E4F0744078000202F19031
:1002E8000AB37401F074007802900ACEF0C8A3F043
:1002F800C8900AD5F0C8A3F0C890E625F0C8000059
:100308000090E624F0C8F5358836C207C208D2E85E
:1003180043D820538EF85391EF90E600E054FDF057
:1003280090E6687408F090E65CE04409F00000008C
:1003380090E61274A0F090E61474E0F0E490E610F1
:10034800F090E611F090E613F090E615F090E618BC
:100358007400F000000090E619F000000090E61B21
:10036800F000000090E61A740C200D027404F000EE
:10037800000090E6917480F000000090E69174808F
:10038800F000000090E6917480F000000090E69183
:100398007480F000000090E65E7440F0D2AF90E602
:1003A80080E04402F0758901758810D2A92290E690
:1003B80080E04408F0F0E04402F07FDC7E0512069D
:1003C800B990E680E054F7F07E187FFF1206AB2064
:1003D8000606DFF8DEF680D62290E6B9E0700B90CC
:1003E800E6B8E024DF700002042C147003020498BD
:1003F80024FE70030204F324FB70030205651470E5
:10040800030205761470030205921470030205A115
:100418002405700302063790E6B8E030E6030205CB
:0D042800B602067B90E6B8E0247F60231446
:1004350060302402705AA205E43325E0FFA200E4EF
:10044500334F90E740F0E4A3F090E68B7402F0029E
:100455000682E490E740F0A3F090E68B7402F00288
:10046500068290E6BCE0F45480C4FFE05407200106
:1004750002701D2F25E024B4F58275837FE054FEBC
:1004850090E740F0E4A3F090E68B7402F002068258
:1004950002067B90E6B8E024FE6007240260400275
:1004A500067B90E6BAE0704390E6BCE0F45480C465
:1004B500FFE0540720010270322F25E024B4F582B5
:1004C50075837FE4F090E6BCE05480131313541F4A
:1004D500FFE054072F90E683F0D2E5F00206829004
:1004E500E6BAE0B40105C20502068202067B90E683
:1004F500B824FE60072402605802068290E6BAE03E
:10050500705B90E6BCE0F45480C4FFE05407200122
:100515000270D82F25E024B4F58275837F7401F02D
:10052500C083C08290E6BCE05480131313541FFFB0
:10053500E054072F90E683F0D2E5F0D082D083EF28
:1005450020E407A37401F0020682E0D2E1F002067E
:100555008290E6BAE0B40105D20502068202067B66
:1005650090E740E4A20133F090E68B7401F00206B7
:0A0575008290E6BAE0600BB40110BA
:10057F00D20112068C020682C20112068C0206827A
:10058F0002067B90E740E530F0740190E68BF002B5
:10059F0006822001030205B390E6BAE0F530120699
:1005AF008C02068202067B90E6B9E0B41028E43094
:1005BF000B0E90E6BCE0F9C3E53399E44002E53455
:1005CF0090E740F0A3E533F090E68AE4F090E68BF5
:1005DF007402F0020682B4114990E6BCE0B53335DF
:1005EF00E5567015E533120D15602A7403121026A7
:1005FF00755604121030120927121041E4900B3E69
:10060F007D40C0E0121117EFF0A3EEF0A3D0E0048D
:10061F00DDF012104590E6B3740BF0A3743EF002B8
:10062F000682B4120002068290E6BBE024FE60143C
:10063F0014601E2402703590E6B3740AF0A374A6FA
:10064F00F002068290E6B3740AF0A374B8F00206C3
:10065F008290E6BAE023F9900AD893C90493C9901F
:10066F00E6B3F0A3E9F002068202068290E6A0E06C
:10067F004401F090E6A0E04480F0C2062290E683A9
:10068F00E47F08F0D2E5F0C2E505E0DFF67F0874FD
:10069F0010F0D2E5F0C2E505E0DFF6227586009096
:1006AF00FB50A3E582458370F9228E318F32E532FC
:1006BF001532AE31700215314E6004D1AB80EF228E
:1006CF000557C0E0E5586005147000F558D0E032CA
:0406DF00C0E0C08334
:1006E300C082C085C084C086C0D074EF529190E6AA
:1006F3005D7401F090E6B8E0B42117A3E0B4FF12F3
:10070300120A54120BC375816F51B9D18212072596
:1007130021E1D206D0D0D086D084D085D082D083B8
:10072300D0E032C0E0C083C082C085C084C086D21E
:10073300045391EF90E65D7408F00000000000D0D0
:1007430086D084D085D082D083D0E032C0E0C0830D
:10075300C082C085C084C0865391EF90E65D74105B
:10076300F0D086D084D085D082D083D0E03253912C
:10077300EFF5A105593232754D00754E00754F00E6
:10078300300B0BE5567019E533120D157005740126
:100793000207AC7403121026121030318412092799
:1007A300755604120BC012093DF54C300A4220095C
:1007B30003120863300D1B90E6AFE0F990E6B0E05A
:1007C300F849600BE5AA20E6FB90E6487406F002C0
:1007D3000835E54D454E605AC333F9E43390E69846
:1007E300F090E699E9F090E6A5E030E2F9020835E9
:1007F30020093FAD48AC49754800754900E4C54F31
:10080300C333F9740033F8496006748090E691F0BD
:10081300EDC399FDEC98FC40194D601690E6A3E0FA
:1008230020E2F990E690E0F890E691E0F97480F028
:1008330080DED208C20712083D2290E6A5E05409E3
:07084300701DC20890F800CF
:10084A0079407F0DE7F009A3DFFA90E698E4F0908B
:10085A00E699740DF0120BC322AC48E549C313CCD8
:10086A0013FD74003400F5481211B9754900227558
:10087A009A0A759B8790E67BE0B45528E0B4532426
:10088A00E0B44220E0B4431C79447F04E0F709DF76
:10089A00FB7F04D209E0F76002C20909DFF7E0A290
:1008AA00E7920A22C20790E6A5E04401F090E6A387
:1008BA00E04401F022E5AC30E1FB90E6047480F0FC
:1008CA000000007402F00000007400F000000074E0
:1008DA008090E691F000000090E691F00000009010
:1008EA00E691F000000090E691F022E533120D1532
:1008FA00602A1210417437900B2E7D04C0E0121149
:10090A0017EF70027430F0A3A3EE70027430F0A3F4
:10091A00A3D0E004DDE6121045120D2722740679F1
:10092A00A0120F5F74017900120F5F740E7908121A
:10093A000F5F221201847407120F5754886009E569
:10094A0056740170EE740122740479FF120F5F74F9
:10095A000579FF120F5F740779A0120F5F120184E5
:10096A007407120F5754806009E556740170EE74CB
:10097A0001221201847407120F5754087009E556B0
:10098A00740170EE740122900A967E067F00120F9F
:10099A00E112018412100C701A740E120F575408C7
:1009AA007007E55670EB7401227402120F57146037
:1009BA00C180DE7407120F577402120F5754037066
:0A09CA0008120A1A1212A380C814C2
:1009D40070057402020A1914702F30092474041269
:1009E4000F57FC7405120F57C313CC13FD7F00126D
:1009F4000F79DDF9EC60A01C80F3809B7402020A7D
:100A040019120A1A1211B9808E7407120F57540161
:100A14006003000000227404120F57FC7405120FC7
:100A240057FDD20975F0007948E7C39C42F0F709F5
:100A3400E79D42F0F709E7940042F0F709E79400D4
:100A440042F0F7E5F06002C209EDC313CC13FD22B6
:100A5400300B2EE556602A7407120F5724B060211C
:100A6400740E790C120F5F1206AB740E7908120F14
:100A74005F780079007407120F5730E704D9F6D86D
:030A8400F4222237
:100AA6001201000200000040C90A00000000010215
:100AB600030109022000010100C0320904000002FE
:100AC600080650000705860240000007050202409E
:100AD60000000AE00AE40B040B2C040309042003BB
:100AE6004D006900630072006F00200053006F0024
:100AF6006C007500740069006F006E0073002803B7
:100B06004200410043004B005000410043004B00AF
:100B160020005500530042003200200043006100CF
:100B260062006C00650012033000300030003000B7
:080B36003000300030003000F7
:100BC000D28522C28522B2852290E6007410F09070
:100BD000E60174C0F090E6C3743FF090E6C2743F43
:100BE000F090E6F37440F075B3FF75B5F075B2EFB1
:100BF000120BC375B4FF75B6FF120C852290E60187
:100C000074F2F075B54090E6C2743FF090E6C3749C
:100C100038F090E6C17400F090E6C074E4F090E61D
:100C2000F5F02290E60174C0F090E6C3743FF090B6
:100C3000E6C2743FF075B5F02204010157001101BE
:100C40005300010053003F035300040103570011F8
:100C5000035300130357003F0757000401015700D7
:100C600011015300010257001F01570006010357ED
:100C7000001303573F220353002303560027035753
:100C8000003F03570090E60174C2F07592E4787F4C
:100C90007980E4F218D9FC75921A78007980E4F230
:100CA00008D9FC900C3975921A78007904E0A36099
:100CB00013FA7B04E0A3F2E82408F8DBF7E8C39416
:100CC0001FF8DAEEE8242054E0F8D9E1787F797F44
:100CD0007A8075921AE360047592E4F21819DAF2D8
:100CE000787F797F7A8075921AE3FB7592E4E2C38C
:100CF0009B6004EBF280E91819DAEB90E6F5F090CE
:090D0000E60174C0F075920022B6
:100D0900C20DE534C3940E4002D20D22F533120D03
:100D19005274004008300D03120BFD740122300D8E
:100D290003120C23120DC722F533120D5250080578
:100D390033E53370F5D322121014F534300D031254
:100D49000BFD120D27E533C32275B00075906212B1
:100D59000DC6759070120DC6E533F590120DC6F4E7
:100D6900F590120DC6D2B7120DC643B070120DC65A
:100D7900759004200D03759003120DC67470F5B0BB
:100D8900120DC67450F5B0120DC6E5B0540F300DF2
:100D990006B40C27020DA3B40B217470F5B0120D23
:100DA900C6E5B0540F300D08B4031074B0020DBE7F
:100DB900B4040874F0F5B0C3020DC5D32222300D76
:100DC90003D2B62275B000227558FAE5BB20E70AAE
:100DD900E55670F774FF90E6F5F07558002280E843
:100DE900E5BB30E7F9227532FFE5BB20E723C0E018
:100DF900D0E0C0E0D0E0C0E0D0E0C0E0D0E0D53243
:100E0900E874FF90E6F5F090E698EEF090E699EF39
:100E1900F022300D29C083C082C085C084C086C03D
:100E2900E090E6F37440F0D0E090E6F1F0000000C5
:100E3900120DD1D086D084D085D082D08322F5906E
:100E4900B2B522300D29C083C082C085C084C08656
:100E5900C0E090E6F374C0F0D0E090E6F1F0000055
:100E690000120DD1D086D084D085D082D08322F5CE
:100E790090B2B622300D23C083C082C085C084C021
:040E89008690E6F178
:100E8D00E0000000120DD190E6F2E0D086D084D0C3
:100E9D0085D082D0832275B300B2B6C2B4E590D2AC
:100EAD00B475B3FF22300D2BC083C082C085C084C2
:100EBD00C086058690E6F1E0000000120DD190E6A7
:100ECD00F2E00586F0A3DFEAD086D084D085D0820B
:100EDD00D08322E583F59AE582F59B75B300C2B404
:100EED00B2B61F120DC6E590F59CB2B6DFF5120D28
:100EFD00C6E590F59CD2B475B3FF22C083C082C005
:100F0D0085C084C086300D27058690E6F374C0F049
:100F1D000586E0A3058690E6F1F0000000120DD1E4
:100F2D000586DFE4D086D084D085D082D08322E5BB
:100F3D0083F59AE582F59BE59CF590B2B6DFF8D086
:100F4D0086D084D085D082D083224440120E1B02DD
:100F5D000E7D4460120E1BE9020E4C4400120E1B56
:100F6D00020E7D4420120E1BE9020E4C74E1120E8E
:100F7D001BEF4440120E1B120E7DCF4440120E1B70
:100F8D00120E7DFE74C1120E1B2274E1120E1BEFA8
:100F9D004460120E1BED120E4CEF4460120E1BEE50
:100FAD00120E4C74C1120E1B227428120E1BEE234E
:100FBD00FE120E4C7400120E4C7400120E4C74E99D
:100FCD00120E1BEF4440120E1BEEFF120EB274C92F
:100FDD00120E1B227428120E1BEE23FE120E4C74E1
:100FED0000120E4C7400120E4C74E9120E1BEF44DD
:050FFD0060120E1BEE66
:10100200FF120F0874C9120E1B227400120F6854CB
:1010120001227401120F68543F227401120F6854A6
:10102200C023232254030303F97401020F702274B4
:1010320006020F68C0E0F97406120F70D0E0227445
:101042000880F1740080ED121031440480E6121021
:101052003154FB80DF12104912108660FB80EFC012
:10106200E0C0F0540160027402F5F012103154FC39
:1010720045F0121036440112103654FE121036D0CA
:10108200F0D0E0227400120F685440600274012212
:1010920012104974011210611412106112106104CD
:1010A200121061121061121061121061121061129D
:1010B20010611210502212104974011210611412A0
:1010C200106112106112106112106112106112107F
:1010D2006112106112106112105022C0E012104908
:1010E200740112106174001210617401121061D047
:1010F200E02323237B0612106123DBFAEE7B082315
:10110200121061DBFAEF7B0823121061DBFA121076
:101112005012105722C0E0121049740112106112CD
:10112200106114121061D0E02323237B0612106198
:1011320023DBFA7B08C0E0740012106112108613E0
:10114200D0E033DBF0FE7B08C0E0740012106112C5
:10115200108613D0E033DBF0FF1210502212104938
:1011620074011210611412106112106104121061E4
:1011720014121061121061121061121061121061CA
:1011820012105012105712104974011210611412E9
:1011920010611210611210610412106112106112BA
:1011A20010611210611210617B1014121061DBFBCE
:1011B200121050121057227428120E1BEDC333FF67
:1011C200EC33FEEF120E4CEE120E4C7400120E4C6B
:1011D20074E9120E1B7440120E1B300D2090E6E3D0
:1011E2007400F090E6D0EEF090E6D1EFF090E6E4F5
:1011F200E0000000120DE774C9120E1B2275B30045
:10120200C2B4ED4C700BD2B475B3FF74C9120E1B8D
:1012120022E54D254DF8E54E354EC82400F59BE8F4
:1012220034F8F59AE536C313F8E53513C3954DF94D
:10123200FBE8954EF8FAEDC399EC984009754D001C
:10124200754E00021254EDFB254DF54DECFA354E6C
:10125200F54EEDC39BFDEC9AFCB2B690E6A5E020FC
:10126200E3FCEBC39401FBEA9400FA4B6014E590B3
:10127200B2B6F59CE590B2B6F59CDBF2EA60031AD1
:1012820080ECE590B2B6F59CE590F59CE54D454EB7
:10129200700C90E698E536F090E699E535F002128A
:1012A200047428120E1BEDC333FFEC33FEEF120E53
:1012B2004CEE120E4C7400120E4C74E9120E1B749A
:1012C20060120E1B300D3290E6D37400F090E6D01F
:1012D200EEF090E6D1EFF07400F5BB00000075323D
:1012E200FFE5AA5401700790E691F0000000E5BB0B
:1012F20030E7EE74C9120E1B22E54F602BFAE59F10
:10130200F590B2B600E59FF590B2B600DAF07480BF
:1013120090E691F074F0F59D7400F59EEDC3954F43
:10132200FDEC9400FC754F0074F0F59D7400F59E81
:10133200EC604B7A4090E6A3E020E2FCE59FF5905A
:10134200B2B6E59FF590B2B6E59FF590B2B6E59FCD
:10135200F590B2B6E59FF590B2B6E59FF590B2B6BC
:10136200E59FF590B2B6E59FF590B2B6DACE7480FD
:1013720090E691F074F0F59D7400F59EDCB5ED6099
:101382003990E6A3E020E2FC90E690E0C313FA90E5
:10139200E691E013C39DF54FE59FF590B2B600E5E7
:1013A2009FF590B2B600DDF0E54F700E748090E6C6
:1013B20091F074F0F59D7400F59E74C9120E1B2213
:00000001FF
